:10000000C02300202D01000029010000290100006B
:1000100000000000000000000000000000000000E0
:1000200000000000000000000000000029010000A6
:10003000000000000000000029010000290100006C
:100040002901000029010000290100002901000008
:10005000290100002901000029010000FD1D000008
:1000600029010000290100002901000029010000E8
:10007000290100000000000000000000290100002C
:1000800029010000290100002901000029010000C8
:10009000290100000000000000000000290100000C
:1000A00029010000290100002901000029010000A8
:1000B0000000000010B5064C2378002B07D1054B3B
:1000C000002B02D0044800E000BF0123237010BDC4
:1000D0006800002000000000E42C0000084B10B570
:1000E000002B03D00749084800E000BF0748036819
:1000F000002B00D110BD064B002BFBD09847F9E731
:10010000000000006C000020E42C0000E42C000043
:100110000000000010B5024B9847024B984710BDF5
:1001200069030000852B0000FEE70000F8B52A4AAD
:100130002A4B9A4211D01A00294B9A420DD2294AD1
:1001400003339B1A9B0801339B000022234822495A
:100150008C58845004329A42FAD1234A234B9A4253
:100160000AD2D34321495B1803218B4304339B18E4
:10017000002102C29342FCD11D4AFF211D4B8B433B
:100180009360FD3990235B001B4AD1501B4AD37802
:100190000325AB4302242343D370D3780C27BB43FE
:1001A00008263343D370164B987B3022904320228D
:1001B00010439873997BB943314399739A7BAA434F
:1001C00022439A730F4A536880210B4353600E4BAE
:1001D00098470E4B9847FEE7E42C000000000020F3
:1001E000680000200400002068000020BC030020FC
:1001F00000ED00E0000000000070004100500041F0
:100200000048004100400041912B000039200000CF
:1002100030B50E4B5622995C0125A9430124214398
:10022000C9B299543B20195C473A91430D3A1143A6
:10023000195457215A5CAA432243D2B25A541A5C29
:1002400048390A4011310A431A5430BD0044004174
:10025000044A136A20210B431362034A034B5A805A
:100260007047C0460004004017400000000C0040EA
:1002700010B5054B9847002204490548054B98479F
:10028000054B984710BDC0465102000000140042C3
:10029000B00300208504000011020000F0B5C6463E
:1002A00000B5C024E40580225204A2601A4B8027C6
:1002B000FF059F621949996262615820195C042206
:1002C000904691431954195C0126B14301252943F5
:1002D000C9B219541C38195C0B329143093A1143C5
:1002E000195480218904A1609F620D4F9F62616152
:1002F00059215C5C424694435C545A5CB2432A43A5
:10030000D2B25A541A5C4A390A4051310A431A543B
:1003100004BC9046F0BDC04600440041000100C04E
:10032000000200C0064BDA6920210A43DA615A69EB
:1003300020310A435A61034A034B5A807047C04632
:100340000004004006400000000C004010B5034BC4
:100350009847034B9847034B984710BD250300006F
:10036000410700009D02000010B5034B9847034B66
:100370009847034B984710BD010B00007102000025
:100380004D030000EFF31083036072B6BFF35F8F7D
:100390007047BFF35F8F036883F3108870470000D6
:1003A000F8B5CE46474680B504000F0090460028B9
:1003B00026D0002926D01000431E9841F122124970
:1003C000124B98470834124D2000A8470028FBD054
:1003D0000026104B99460E4DB95D2000C8472000FD
:1003E000A8470028FBD001364645F5D30A4D20002A
:1003F000A8470028FBD030000CBC90469946F8BDB9
:100400000020DBE70020D9E7FC2B0000950A000064
:10041000710C0000610C00007B0C0000F8B5CE46AA
:10042000474680B504000F00904600281DD00029E3
:100430001DD01000431E9841862252000D490E4BDC
:100440009847002608340D4D0D4B99462000A847CB
:100450000028FBD02000C847B85501364645F5D3E3
:1004600030000CBC90469946F8BD0020E4E700201F
:10047000E2E7C046FC2B0000950A0000850C000056
:10048000690C000070B505000C00002813D00800AE
:10049000431E9841C0B234220849094B98472800AE
:1004A00008302100074B9847002803D1064B6B60AA
:1004B000064B2B6070BD0020EDE7C046FC2B000012
:1004C000950A0000350C00001D040000A103000087
:1004D000F0B504000E4B5A78904217D0002300204C
:1004E0000B4F0F2626403D0008E0013040B20428A3
:1004F0000AD02033EA185278A24206D0D95D0029EA
:10050000F3D19642F1D100E00538F0BD0020FCE7C0
:10051000840000200020704770B504000D000A4BD5
:1005200098474201094B9B189A780023032A01D06F
:10053000180070BD4001054B181883692900200080
:1005400098470300F4E7C046D1040000840000206F
:10055000F0B585B005000F001600514B9847040018
:10056000002F62D14F4B420199180020C870D35C14
:10057000002B0ED062014B4B9B1801229A70640134
:10058000484B1C19E178E36932002800984705B010
:10059000F0BD8B78032B0CD0424B62010C329A18C1
:1005A00064011C1960780021E36998470223A37055
:1005B000EDE73C4A0B000C254D5761010C315218F8
:1005C0005878DB6901219847002817D06201354B24
:1005D0009B1805229A70033ADA70002D09DB64013A
:1005E000304B1C1960788023184301212E4B98470B
:1005F000CDE764012B4B1C196078F6E76401294BA9
:100600001C190423A3706378002201920292002D2A
:1006100008DB8032134301A8037201234372234B8A
:100620009847B4E70F221340F5E7012F0AD0022FB5
:100630001DD0032F2CD042011A4B9B1806229A7012
:10064000DA709CE7174B420199180220C870D35CFE
:10065000002B05D06201134B9B1805229A708EE780
:1006600002228A70002128000F4B984787E70D4B24
:10067000420199180420C870D35C002B05D0620198
:10068000084B9B1801229A7079E702238B707EE752
:100690004201044B9B1800229A700532DA706EE713
:1006A000D104000084000020C1190000951B000047
:1006B000F0B5C64600B504001D4B9847060045013D
:1006C0000C351C4B5D19290020001B4B9847C0B20C
:1006D00008280AD001212000184DA8478020204377
:1006E0000121A84704BC9046F0BD00212000134B17
:1006F000984698478027274300213800C047720159
:100700000C4B9B1801229A705B69290020009847C6
:100710000028E7D17601074B9E190523B37001210C
:100720002000064CA04701213800A047DAE7C04668
:10073000D104000084000020251B0000C119000026
:1007400010B5104B984700281BDB0F4C802200216E
:1007500020000E4B984723008034FF210C4A59702B
:100760005A619A61DA612033A342F8D10949002025
:10077000094CA04709490120A04709490220A04788
:10078000002010BDA113000084000020EB2B00000E
:1007900015050000B1060000CD1D00001905000080
:1007A0005105000010B5014B984710BDA91D000070
:1007B00010B5014B984710BD7D14000010B5014BDA
:1007C000984710BDCD14000010B5014B984710BDDF
:1007D000DD140000F8B505000E0017000F4B984718
:1007E000002814DAFF200D4B9847041E12DB3A0054
:1007F000310028000A4B9847002807DB094A6401AA
:1008000013195D7003231E40A6540020F8BD142068
:100810004042FBE715204042F8E7C046D104000003
:10082000ED1400008400002010B582B200210020E9
:10083000014B984710BDC046D507000070B50500B4
:10084000064B9847041E07DB2800054B98476401B8
:10085000044B1C19FF23637070BDC046D104000017
:10086000191600008400002070B504000E4B984754
:10087000051E15DB43010D4A9B5C5A42534101336F
:1008800041010A4A521893702000094B98470028EA
:1008900000DB70BD6D01054B5D190023AB70F8E7FF
:1008A00012204042F5E7C046D10400008400002039
:1008B000E5160000F0B5D6464F464646C0B586B0B0
:1008C0000400077A3800404B98470500667A636851
:1008D0009846002800DA71E004A83C4B98476A016A
:1008E0003B4B9B189A7817236B441A701B78012B8B
:1008F00010D004A8374B984717236B441B78DBB202
:10090000052B5ED0062B23D00120002B3CD11320D9
:10091000404239E02E4B99466B019A464B46534470
:1009200003229A7004A82B4B98474B465246D35C3F
:10093000002B10D0237A721E9641F6B222680192E3
:10094000424602927FB2002F17DB0F22134016E0BF
:100950001020404218E06B011D4AD218D17C0902D8
:10096000937C5B189BB2002B14D10423937000225C
:100970000126237A2168019102928022134301A863
:1009800003724672144B984706B01CBC90469946B9
:10099000A246F0BD42469A4200D91A006D010C49A8
:1009A0004D19297B7F2905D8237A2168019102926C
:1009B0000026CAE79A42B6417642DAE71220404260
:1009C000E2E70220E0E7C046D10400008503000012
:1009D0008400002093030000951B000070B5040004
:1009E000002905D0012921D00221134B984770BD61
:1009F000124B9847051E1CDB022120000E4B984726
:100A00000028F4D0002120000B4B98470028EEDB93
:100A10006D010B4B5D190123AB700233EB70EB6979
:100A200000220321200098470020E0E7024B98476E
:100A3000DDE712204042DAE7C1190000D1040000CE
:100A40008400002070B50D0014000F4B9847030080
:100A5000221E08D0002B05DB012D0BD0002D04D069
:100A6000022D0CD070BD094AF4E74001084B18185C
:100A70004261F7E74001064B18188261F2E7400136
:100A8000034B1818C261EDE7D10400001505000002
:100A900084000020002800D100BE70470368002BAE
:100AA0000AD08B420AD01B68002B03D09942FAD19E
:100AB000012000E0002070470020FCE70120FAE759
:100AC00070B505000E0004680A4B98470123584092
:100AD000C0B24F220849094B98472B68002B03D11D
:100AE0002E60336005E01C002368002BFBD12660DC
:100AF000336070BD9D0A0000182C0000950A0000AC
:100B000010B5084A536804210B435360064B9847BD
:100B1000064B98470220064CA047064B9847FD20FD
:100B2000A04710BD00400041790B0000910C00006F
:100B3000390B0000B90C0000C30709D50B4B80220C
:100B400052009A600A4A5A601A005378DB09FCD1B5
:100B5000830709D5054B0222FF329A60054A5A6085
:100B60001A005378DB09FCD17047C046000C0040E6
:100B70000007010001050100064B1A7AD2B21A7271
:100B80005A7AD2B25A729A7AD2B29A72DA7AD2B2C5
:100B9000DA7270470004004010B504001F4BC31800
:100BA0009B0ADBB2032B04D01D4A1E4900201E4BBA
:100BB0009847E369DB0718D40322E3691A42FCD1A2
:100BC00023689B070BD523680222934323600132DD
:100BD000E3691A42FCD10222E3691A42FCD10523DF
:100BE00023600322E3691A42FCD10122E3691A421D
:100BF000FCD10E4B23600322E3691A42FCD1C023CF
:100C00009B0263600722E3691A42FCD1084BA3816F
:100C10000023A3733022A354002010BD00F8FFBDB1
:100C20003A020000382C0000950A00000400104031
:100C30002BF6FFFF70B505000C00431E9841C0B2B3
:100C4000B4220449044B98472C602000034B98477A
:100C500070BDC046382C0000950A0000990B0000BA
:100C6000036889B2198570470368188DC0B2704750
:100C70000368187E0123184070470368187E8007B8
:100C8000C00F70470368187E4007C00F7047000010
:100C9000084B0E229A829A6902210A439A611A7FAE
:100CA0001D310A401A7719000222CB681A42FCD083
:100CB0007047C046000800408222D201174B5A807C
:100CC0000222174B9A8419000E32CB681A42FCD0CC
:100CD000134B144ADA62FC22D2019A62124A9A84B5
:100CE0009B8C5B0714D50E49D022CB681340D02BC8
:100CF000FBD10B4A938C80210B439384074A537892
:100D0000DB09FCD1064A936902218B43936170474A
:100D100003491022CB681A42FCD0EAE7000C0040DD
:100D200000080040B90501040608000000207047D3
:100D300070B5837C0F221340C17C083A0A40012A17
:100D40000BD05A0119498C4662441021D1715B01C4
:100D5000174A94466344197070BD4A060ED5C27C8A
:100D600040218A43C2745A01124CA4466244802531
:100D70008224640015550624FF341155C27C0821D5
:100D80008A43C2740C495A018C180025A572A576B5
:100D90001300064CA44663446F24DC71044B9C464C
:100DA00062441470807C8B6E9847D5E700510041F7
:100DB00008510041005000410401002010B52022DC
:100DC0008A40D2B2817C0F230B405B0105498C46DF
:100DD00063441A708268807C034B1B6F0121984723
:100DE00010BDC046085100410401002010B5837CAD
:100DF000FF2B02D0C27C520600D410BDC27C40241E
:100E0000A243C27482680248046F1800A047F4E746
:100E10000401002030B583B0837C01AC252525700A
:100E200025356570FF2B1BD0C47C640618D50F24B4
:100E30002340002916D05C010E4DAC466444802549
:100E4000257101AC645C59010A4DAC466144CC711A
:100E50005B0109498C4663441C701100074B98479D
:100E600003B030BD5C01034DAC4664444025657160
:100E7000E7E7C0460051004108510041ED0D000078
:100E800070B582B0837C0F22134001AA0424147031
:100E9000043454705D01002931D01A000832520127
:100EA000324C145D6406640F0A015219304DAA18C1
:100EB000957AEDB2022C2AD0AC0741D5C57C947A44
:100EC0000226B443947201AA545C5A01294EB446D6
:100ED0006244D4715B01284A944663441C70072322
:100EE0002B40012B3FD1C37C5B063CD5C37CDB0987
:100EF000994238D000221900204B984733E01A005D
:100F000008325201194C145D07221440CCE7EC075B
:100F1000D2D5947A0125AC43947201AA545C5A014B
:100F2000144DAC466244D4715B01134A9446634449
:100F30001C704B1E9941C9B20422104B984712E015
:100F40005A00521812010A4882180020907201AA11
:100F5000515C5A01074884466244D1715B01064ADC
:100F600094466344197002B070BDC0460050004101
:100F7000040100200051004108510041150E0000FD
:100F8000F0B5C64600B50C4D2C0074342935FF353C
:100F90000A4B9846FF27002603212000C047A7746C
:100FA000E6741434AC42F7D1602200210248044BAD
:100FB000984704BC9046F0BD04010020ED0D0000F0
:100FC000EB2B0000F0B5C64600B504000E00837C94
:100FD0000F251D40002900D1AAE06A015A4B9B1839
:100FE00058698004800C238A584A934200D19AE0C1
:100FF000013B9AB2E37C07271F40002E05D06B010E
:1010000053498C4663440221D971A368C118A16079
:10101000636899424AD25B1A9BB2E27C920635D54C
:10102000228A101C92B29A4200D9181C83B29846A8
:1010300023689C4661444246E068464B9847E16815
:101040006A01414B9B1819616A013F4B9B185A6911
:1010500041468904890C920B92030A435A615A69EA
:101060003D490A405A61002E07D1012F59D04A222A
:101070006B013A498C4663441A706D01344B9C46AF
:10108000654480236B7104BC9046F0BD1A1C80201F
:101090008001834201D9324B1A8893B29846236863
:1010A00059186A01284B9B181961CDE7E37CDB06D0
:1010B0000FD5E37C10229343E3746A01224B9B1803
:1010C0005A69920B92035A615A6923490A405A613C
:1010D000C9E7012F0ED06D01224B9C4665444A237F
:1010E0002B70218A024091420BD0002120001E4B20
:1010F0009847C8E76D011B4B9C4665444B232B70FA
:10110000EFE7E37C40229343E374A07C0E4BDB6E5D
:10111000A16898470028B6D1E37C40221343E374CA
:10112000E3E74E22A4E7E77C07231F40074A66E770
:10113000038A064A0020934200D059E7E37C072740
:101140001F400020014A60E704010020FF03000067
:1011500000510041D92B0000FF3F00F00951004130
:10116000542C000008510041ED0D0000F8B5DE469A
:1011700057464E464546E0B504008846837C0F2519
:101180001D40002957D06A017D4B9B185A681201F7
:10119000920C92465F68BF04BF0CBB46068A794B2F
:1011A0009E4200D1CDE0013EB6B25F463740E37CBF
:1011B00007221A4091464346002B05D06B01724A24
:1011C000944663440122DA71E37C9B060FD5636881
:1011D000002B39D0A0681B1A9BB222689446604449
:1011E000E1681A00BB4200D93A00684B984763682F
:1011F000002B29D04246002A42D0228ABA423FD947
:10120000E37C10229343E374A3685B44A3604B46E2
:10121000012B00D187E06B015D4A9446634425228F
:101220001A70002D02D1564BE2681A60002120008E
:10123000584B984759E0068A524B9E4200D18EE0A7
:1012400000239B469A46AEE7E37CDB0600D47FE0B2
:10125000E37C1022934320221343E374484A6B013A
:10126000E1689950218AD3185A68890409094A48C3
:1012700002400A435A605A68920B92035A6022E075
:10128000A2685244A2609342C1D99B1A9BB2E17CEE
:10129000890630D5228A111C92B29A4200D9191CB3
:1012A0008BB2E0686A01364950506A0134498918A6
:1012B0004A689B041B093848024013434B604B6843
:1012C0009B0B9B034B604346002B08D125224B46CA
:1012D000012B2FD06B0131498C4663441A706D018C
:1012E000294B9C46654440232B713CBC9046994653
:1012F000A246AB46F8BD218A8B420AD980218901DA
:101300008B420DD8B34321688A1869011C480A50E2
:10131000CBE78B42F7D2E17C20200143E174F2E776
:1013200080239B01EFE76B01194A944663442D2209
:101330001A7076E76A01124B9B1800229A762D32BA
:10134000C8E7BF05BF0DC37C07221A40914635E7A9
:101350004346002B0CD1A3685344A36057E7C37CDA
:1013600007221A409146002700239B469A462BE706
:10137000238ABB4200D943E7A3685344A36046E7EE
:1013800004010020FF03000000510041D92B0000A0
:1013900008510041ED0D0000FF3F00F009510041F0
:1013A00010B5314B9B78DB071FD42F4903228B7874
:1013B0001342FCD12C4B1B789B070ED52A4A13787D
:1013C00002218B431370110003228B781342FCD14E
:1013D000254902228B781342FCD10122224B1A703C
:1013E000190002328B781342FCD11F4901228B78FD
:1013F0001342FCD11D4B1E4A1A665A669A66DA667B
:101400001A671C4B98471C4B1B685A0B1F210A403C
:10141000980C01409B015B0F1F2A1FD01F291FD072
:10142000072B1FD092010A431B0313430E4A138557
:10143000D37803210B43D370D3780C210B43D370A3
:1014400004231370110003228B781342FCD1064B46
:10145000064A5A6201221A81002010BD1A3ADDE7BD
:101460000239DDE7023BDDE70050004104010020C6
:101470002D0D0000810F000024608000104B9B7830
:101480009B071AD10E4903228B781342FCD10C4BD7
:101490001B78DBB29A0708D402221343084A137060
:1014A000110003228B781342FCD18022054B1A6075
:1014B000054A034B1A830020704711204042FBE786
:1014C0000050004100E100E08D020000024A138953
:1014D00001218B4313817047005000418023184342
:1014E000014B98727047C04600500041F0B50F2480
:1014F000044043B29C46002C54D02500002B07DB4F
:10150000032319402700022C50D91220404225E025
:10151000A51CF5E76346002B21DB7B00DB199B0054
:101520003B4C1B59002B66D17B00DF19BF00384BA9
:10153000FF58384BAE007419A4001C198034276082
:1015400060337419A4001C19A2842734013121705E
:101550007519AD005B19263318700020F0BD7B00B3
:10156000DB199B002A4CE3185B68002B06D17B003B
:10157000DF19BF00264BDF197F68DAE77B00DB1934
:101580009B00234CE3185B899342F0DA132040421E
:10159000E4E714204042E1E714204042DEE7132054
:1015A0004042DBE70323194000250027AB005B190D
:1015B0009E00184B9B1986331B78FF2BE9D100291D
:1015C000A8D1002C04D06346002B01DB0234E4B226
:1015D000A3001B199B000F4CE41886342378FF2BC3
:1015E000DAD17B00DB199B00094C1B59002BD6D0AC
:1015F0006346002BB3DB7B00DB199B00044CE31834
:101600001B89934200DB8FE713204042A6E7C046C8
:10161000582C000004010020F8B505000F240440F8
:1016200047B2002C10D02000002F02DB022C02D980
:10163000F8BDA01CFAE706000130830018188000EE
:10164000254B6033181802E0234874300026B3009D
:101650009B199A00204B9B1886331B78FF2BE7D0F1
:10166000F90F03221D4B9847B3009B199A001A4BA0
:101670009B188033DA7907231340012B1BD0002FEE
:101680001FDB6D01164B9C46654480225200AB5C0B
:1016900007218B43AB54104B6033B1008A19920081
:1016A0009A182732002010708E19B6009B19263325
:1016B000FF221A70BCE708356D010022084BEA547E
:1016C000E9E76401064B9C46644480225200A35C17
:1016D00070218B43A354DEE704010020150E0000A7
:1016E00000500041F0B5C64600B50F22024040B29E
:1016F000002A00D192E0130000280BDB1100083211
:101700005201AA4C155DEDB2022900D88DE01220DD
:101710004042E5E0931CF1E776322A4275D1A34AB4
:1017200090464444112080225200A0549A00D218BE
:1017300095009F4A60325219928C95039D4805404E
:1017400080208000824200D9CDE00138FF388242FB
:1017500000D913E1802A00D900E1402A00D915E11F
:10176000202A00D902E1102A00D917E1F838904266
:1017700080414042060735437D609504AD0CB9E0D9
:1017800070222A4244D18A489E00F21892008218A0
:101790008032D2795207520E1543844A94466444EB
:1017A00080225200A5546030F618B6008019808C53
:1017B0008504AD0C0132FF320723904214D8013A60
:1017C000FF3A013B90420FD8013B80280CD8013BE7
:1017D000402809D8013B202806D8013B102803D80F
:1017E000F83A8242924153421B072B437B6180228D
:1017F00082235B00E25449016D4B591800238B761C
:1018000000206DE0122040426AE01420404267E070
:101810001420404264E01420404261E080235B00D9
:10182000624AD55CEDB2002100239A00D2189400E0
:101830005F4A1219863212789446FF2AE2D04C0190
:101840005B4A17199E00F618B60092198032D679B5
:1018500007223240012A00D15EE7002890DB6A07A8
:10186000D9D153489E00F218920082188032D27962
:101870005207520F15434D4A944664448022520049
:10188000A5546030F618B6008019858CAB03494822
:1018900018400132FF320723954214D8013AFF3A2B
:1018A000013B95420FD8013B802D0CD8013B402DC8
:1018B00009D8013B202D06D8013B102D03D8F83A5A
:1018C000AA42924153421B0703437B6040220623F6
:1018D000FF33E2544901364B591800238B72002024
:1018E00004BC9046F0BDE020C00505437D60950432
:1018F000AD0C07200007284378610625FF354026F8
:10190000665582277F008020E0552948490141180B
:1019100000248C728C760F3461460C409900C918F3
:10192000890041188031096863011950C018416865
:1019300092041409204A0A40224342604268920BF2
:1019400092034260194A9A18B021D15556551B4A44
:101950009446634410221A700020C1E7A020C005FD
:1019600005437D609504AD0C0520C3E7C0208005CC
:1019700005437D609504AD0C0320BBE7C020C00586
:1019800005437D609504AD0C0620B3E78020C005BB
:1019900005437D609504AD0C0420ABE780208005F5
:1019A00005437D609504AD0C0220A3E70050004183
:1019B0000401002000C0FF0FFF3F00F0095100416B
:1019C000F0B50F23034040B2C40F002B09D01A001A
:1019D000002804DB022B05D91220404219E09A1C92
:1019E000F8E70022012915D0002936D093009B1872
:1019F0009B00474AD218863212780F2313405B01AE
:101A0000444A9446634498791023A3401840431EE7
:101A10009841F0BD1025A540EDB23D4990008318D6
:101A20009B00CB1886331E780F2333405E01394F5D
:101A3000BC46664475712025A540ECB25B01364D6D
:101A4000AC4663441C70821892008A188032D379A5
:101A500008210B43D3710020DBE793009B1899000A
:101A60002B4B5B1886331B780F210B405D012B49F4
:101A70008C466544832149006E5CF639A140002004
:101A80000E42C6D0C9B20530FF3029542021A140F2
:101A9000C8B25B01224EB446634418700823FF337A
:101AA000EB5C0B4209D00823FF33E854073BFF3BB4
:101AB000A340DBB2822149006B5493009B1899002C
:101AC000134B5B188033D97907230B40012B0BD0C4
:101AD00093009A1892000E4B9B188033DA790821F4
:101AE0008A43DA71002094E70633FF33E95CD63B82
:101AF0000020194200D08CE793009A189200044B02
:101B00009B188033DA7908218A43DA7181E7C0466D
:101B100004010020005100410951004100500041E2
:101B20000851004170B50D000F2318404401164BB9
:101B30001B1919685B689B049E0C02281AD8002D9B
:101B40001BD0124B9C46644480235B00E35C112B4A
:101B500016D10823FF33E35C0020DB0600D470BD00
:101B6000082228000A4B984710220823FF33E2542A
:101B70003000F4E712204042F1E712204042EEE745
:101B800013204042EBE7C046040100200050004112
:101B9000D92B0000F0B5DE4657464E464546E0B527
:101BA00085B08046067A0F23334076B2002B00D1F1
:101BB000D3E01800002E39DB0400734A6032411C68
:101BC0008D006D18AD005519810009188900521853
:101BD000918C6E4A91422BD04F1EBFB24246526842
:101BE0001740022B00D9A4E043461B686848834293
:101BF00020D998180190674884460198604519D803
:101C00009B0717D1002E32DB914200D9AFE0002FA5
:101C100030D0A3001B199A005B4B9B1880331B68C4
:101C2000002B00D18BE0002399460FE0981CC3E7FE
:101C30000F00D3E7A3001B199A00534B9B18803366
:101C40001B68002B00D177E001239946A3001B19E4
:101C50009A004D4B9B188033DB7902201B070CD573
:101C600005B03CBC90469946A246AB46F0BD002369
:101C70009946EBE700239946E8E703A8464B9847C7
:101C8000A3001B199A00404B9B188033DB795B063D
:101C900044D4A3001B199B003B4A93469B448023DA
:101CA0005B449A46DB79402213435246D37103A822
:101CB0003A4B98475B46424612685A67424652681A
:101CC0009A6700235A46D367F20FD2015346D97957
:101CD0007F230B40494649011343202293430B4382
:101CE0005246D37143465B7A0022002B02D07A42DF
:101CF0007A41D2B2A3001C19A400234B1B198033D4
:101D00001201DF7910218F431743DF71002E0ADBA8
:101D100000212800224B98470020A1E703A81F4B71
:101D2000984701209CE7002128001E4B984700207F
:101D300096E71220404293E71320404290E712209A
:101D400040428DE7132040428AE743465A68970590
:101D5000BF0D0D4D7435002446E70B4A6032918C5F
:101D60000A4A9142F1D0084D7435002434E7A300AB
:101D70001B199A00044B9B1880331B68002BE1D081
:101D80000123994662E7C04604010020FF030000DA
:101D9000FFFFFF1FFF7F002085030000930300006B
:101DA0006D110000C50F00000B1E06D0012806D0E3
:101DB000002801D1034A13667047034BF6E7014A36
:101DC0005366F9E7040100202D0D00000B1E08D01A
:101DD000002808D0012809D0022806D1054A136737
:101DE00003E0054BF4E7034A93667047014AD36664
:101DF000FBE7C046040100202D0D0000F8B5824B22
:101E00001E8CB6B2002E03D0804C74340025B9E08D
:101E1000998B1B8B0B405A0717D49A051CD41A06B2
:101E20003ED470221A4244D11A075ED4DB07EBD5A8
:101E3000754B774A9A839A82923AFF3A1A83734B88
:101E40005B6E00210420984705E004226E4B9A83C4
:101E50006E4B1B6E9847F8BD6B4B6D4A9A839A8206
:101E6000923AFF3A1A83694B1B891B071B0F032BFE
:101E70000CD0664B1B8D1B071B0F00216F3A032BE9
:101E800005D0624B5B6E03209847E4E700225201C5
:101E90005E4B9B1819894904490D00221A81F0E70D
:101EA0008022594B9A83594B5B6E0021052098473D
:101EB000D1E7554B9A839A82554A1A83554B9B8C8E
:101EC0009B060CD45349323AFF3ACB681340D02BCF
:101ED000FBD14E4B5B6E002102209847BBE74D497A
:101EE0001022CB681A42FCD0F3E7474B0021802236
:101EF00052009954F83A9A8368329A82444A1A8373
:101F0000454B9847414B5B6E002101209847A2E763
:101F1000CB0607D44B0608D48B062ED500213F4BA9
:101F200098472AE03E4B984727E001213B4B9847D2
:101F300023E04B060ED40B0710D48B0712D40723D3
:101F40001A40012A19D14B0710D4CB0615D5344BB2
:101F5000984712E00121314B98470EE00121314BA7
:101F600098470AE00121304B984706E000212D4BAD
:101F7000984702E00021294B984701351434092D78
:101F800000D168E72000A17CFF29F6D00F230B4089
:101F9000012199400E42F0D05901244FBC466144C2
:101FA000C9795B01224FBC4663441B781940E4D0D9
:101FB000AB005A199200154B9C4662447032D27D98
:101FC00047231340012BA3D053B2002BB1DB8B0668
:101FD000D0D44B070CD4CB070ED407231A40012AC8
:101FE000CBD10B070CD4CB06C7D50D4B9847C4E714
:101FF00000210C4B9847C0E701210E4B9847BCE7E6
:102000000121084B9847B8E7005000410401002027
:102010000102000000080040810F0000BD0D00001B
:10202000310D0000810E0000C50F0000005100417D
:10203000095100416D11000010B5014B9847FEE7B2
:1020400015010000F0B583B006000C0015000A78F9
:1020500053069B0F012B00D06CE0097963791B02BA
:102060000B433B490978994203D039494978994251
:1020700063D152B2002A0EDBA779E3791B021F431A
:10208000344B98476378202B18D0222B3CD00D205E
:10209000404203B0F0BD012D52D06378212B51D1C5
:1020A000A279E3791B021343072B4ED100230722A9
:1020B000274908313000284CA047EAE7072F34D1E0
:1020C000002D1AD0072201006846244B9847204B68
:1020D0001B69002B05D06846984703000020002BA1
:1020E000D7D01B4A1300009991606A4692889A8162
:1020F0006A4692799A730020CBE7002307220100F9
:102100003000154CA047C4E7002300220021002026
:10211000114DA8470E4B5B69002B09D0A278E078DF
:102120000002104398470020B3E701204042B0E787
:102130000020AEE70A204042ABE70A204042A8E771
:102140000020A6E70D204042A3E701204042A0E77F
:10215000EC020020152A0000C5240000D92B000045
:10216000F0B5DE4657464E464546E0B583B016000C
:10217000012968D000290BD0022900D193E00D205D
:10218000404203B03CBC90469946A246AB46F0BDE7
:10219000836898461068002800D187E001930123E6
:1021A00043449B46474F484B9946827843790821E0
:1021B0008B43022B02D00A204042E2E701998A4673
:1021C0000B789A4275D0FF2B76D10A700522716880
:1021D0003E4B9847041E1ED130680378C018042275
:1021E00071683A4B9847019B5B4527D0019B0133AF
:1021F00001930028D9D10A204042C2E753469D707E
:102200002800314B98473460207820187168304B93
:102210009847041EE0D0A57863791B022279D21872
:1022200092B2E1782800B847002848D16BB2002B61
:10223000E4DB43461D712800C847E4E70122254B33
:102240005A7100209DE78468002A08D013685B79E2
:1022500008229343022B02D00A20404291E72378C0
:10226000FF2B08D0FF232370A078FF2803D01A4B40
:102270009847FF23A3706378FF2B08D0FF23637078
:10228000E078FF2803D0144B9847FF23E3702079B0
:10229000FF2803D0104B9847FF23237100220D4BDA
:1022A0005A7100206DE71B2040426AE70A20404235
:1022B00067E71220404264E71C20404261E7142097
:1022C00040425EE7D507000069080000312A00009F
:1022D000672A0000EC0200203D08000010B50A4B00
:1022E000984701280CD80948094BC361006218308F
:1022F000084B984708490120084B9847002010BD1B
:1023000011204042FBE7C046212A0000EC020020D9
:1023100061210000B92900000000002021290000EF
:1023200010B5064B1C69002C07D0002201212000AB
:10233000636898472468002CF7D110BD1003002073
:1023400070B506000D00074BDC68002C03D170BD92
:102350002468002CFBD06368002BF9D029003000E2
:102360009847F5E710030020F8B507000E001500A8
:102370000D4B9C68002C04D1002011E02468002C37
:102380000DD06368002BF9D02A003100380098473F
:10239000002806D00A30F1D00120404200E00020A1
:1023A000F8BD0120FCE7C0461003002010B5064B25
:1023B0005C68002C03D110BD2468002CFBD063683E
:1023C000002BF9D09847F7E71003002010B5140050
:1023D000002903D0012929D0002010BD1378002B3B
:1023E000FAD15378052B11D0092BF5D19278124BE5
:1023F000DA76A378E178090219434B1E994103313B
:102400000D4B997601200D4B9847E5E790780C4BE2
:102410009847A378E178090219434B1E994102318C
:10242000054B99760120054B9847D5E701222100FD
:102430000020044B9847CFE7100300204123000001
:10244000C90700006923000010B50D4B98470D4CDB
:102450000223A3760023E376637700200A4B984794
:10246000207F0A4B98470A4A00210020094CA047C8
:10247000094A02210020A0470020084B984710BDC0
:1024800021230000100300203D080000290800005F
:10249000E1240000450A0000CD2300006908000087
:1024A00010B5002802D0012804D010BD0020034B35
:1024B0009847FAE7024B9847F7E7C04641230000E8
:1024C0004924000010B584B001AC01910292207241
:1024D00063722000014B984704B010BDB50800009E
:1024E000F0B5C64600B584B005000C000022B54B1F
:1024F0009847431C0DD0012301280BD022781F23BD
:10250000110099430BD0CBB2802B00D1F8E000230F
:1025100000E00023180004B004BC9046F0BD6378CE
:102520000B2B00D9E4E19B00A749CB589F46012320
:10253000002200212800A54CA04743424341DBB2C2
:10254000E8E7A278002A1AD0A14B1B6859681868DE
:10255000A04B9847002800D1D4E1C3781B028178B2
:10256000C91889B24118039104229B4B98470290E5
:10257000002806D0FF24964F974B98461AE0974BB9
:1025800098470123002200212800904CA047434295
:102590004341DBB2BEE7340000E034000298037828
:1025A000C0180290039B019304221900C0470290B7
:1025B0000028E6D08678A642F0D03C69002CEAD00C
:1025C00002AA00212000636898470028E5D024680B
:1025D000002CF5D13400E1E71F231A400023022A22
:1025E00098D1A379E27912021A430023002A00D07D
:1025F00090E7207900217A4B98470123002200219F
:102600002800724CA047012384E71F231A400023AF
:10261000022A00D07EE7A379E27912021A4300234E
:10262000002A00D076E7207901216D4B98470123DD
:10263000002200212800654CA04701236AE7A37807
:10264000E5782D021D432379647924021C43604AF6
:102650001368D27E596818685E4B9847002847D0A7
:102660000290C3781B028178C91889B2411803917E
:102670000422594B984700283CD0574E08E0029856
:102680000378C018029004220399B047002833D081
:102690008378A342F3D1C378AB42F0D102904C4B84
:1026A0001E69002E2AD002AA0121300073689847C3
:1026B000002804D03668002EF5D100232AE773687D
:1026C00002AA0021300098470023002800D021E70B
:1026D000002D05D03E490122A2404B7F13434B778A
:1026E0000023002200210020384CA047012311E7DD
:1026F00000230FE700230DE700230BE7002309E782
:102700006378062B33D0D9B2062922D9082B00D101
:10271000AFE00A2B00D0EDE02D4B5A7F2179637991
:102720001B020B431A41D30700D4CAE0284B1D6992
:102730000023002D00D1EDE62200022128006B6865
:102740009847002800DBC8E02D68002DF4D1002355
:10275000E0E6002B00D0CDE01F231A40D3B2012BBE
:1027600000D892E0022A00D19FE00023D2E6A378AD
:10277000E27812021A43130A022B33D0032B56D0ED
:10278000012B01D00023C5E6A279E3791B02134394
:102790001A1C122B00D9122294B20D4B1B685968D7
:1027A000186801220C4B9847002800D1A4E00023B0
:1027B000220001002800054CA04743424341DBB200
:1027C000A8E6C046692300007C2C0000C524000058
:1027D00010030020AD2A0000312A00002123000050
:1027E000DD090000A379E67936021E43464B1F7FC0
:1027F0001B680132D2B259681868444B9847011ED1
:102800007CD0C3781B028478E418A4B20023A642CB
:1028100005D9013F3E4073427341DBB226003200CE
:1028200028003B4CA04743424341DBB272E6A37908
:10283000E179090219430C00334B1E7F1B68D2B2A9
:1028400059681868334B9847011E59D00278002305
:10285000944206D9731E2340180043424341DBB221
:102860001400220028002A4CA04743424341DBB217
:1028700050E6254BDA7E59690A7059690023012216
:102880002800234CA047012344E6002302931E4C5A
:10289000022202A96069204B984761690023022245
:1028A00028001B4CA047012334E6207902211B4B52
:1028B0009847002803DB012318400290E7E7002334
:1028C00028E6114B002259690A7059690023013228
:1028D00000200F4CA04701231CE60B4B5A691070D7
:1028E0005969002301220020094CA047012311E669
:1028F00000230FE600230DE600230BE6002309E684
:10290000002307E6002305E610030020AD2A00009F
:10291000C5240000152B0000D92B0000DD090000A4
:1029200010B5012809D0002802D002280AD010BD15
:1029300007480430074B9847F9E705480830054B2E
:102940009847F4E702480C30024B9847EFE7C0463F
:1029500010030020C10A000070B50400431E984116
:10296000C0B20C4A0C490D4B98470D4B98470028B4
:102970000EDB0C4D2022002128000B4B98476C6188
:102980000A4900200A4CA0470A490120A04700201C
:1029900070BDC04655030000AC2C0000950A000035
:1029A0004107000010030020EB2B0000AD230000C6
:1029B000A5070000A124000010B501000248103056
:1029C000024B984710BDC04610030020C10A00000A
:1029D00010B50B4B9B7E002B0CD100280DD0084B63
:1029E00018600268D2791A7701229A76054B9847C7
:1029F000002010BD04204042FBE709204042F8E7D8
:102A000010030020B107000010B5014B984710BD1E
:102A1000BD070000014B58697047C04610030020F5
:102A2000024B987EC30600D510207047100300208B
:102A300010B5884211D20378012B10D94478944202
:102A40000AD0C018814206D90378012B09D94478ED
:102A50009442F6D100E0002010BD0020FCE70020E9
:102A6000FAE70020F8E7884215D20378012B14D941
:102A70004278042A13D0052A0CD0C018814208D904
:102A80000378012B0DD94278042A0CD0052AF4D101
:102A900000E0002070470020FCE70020FAE700205B
:102AA000F8E70020F6E70020F4E7000070B50C001E
:102AB00015000222164B984700281DD084421CD9CD
:102AC0000378012B1BD94378022B1AD14379AB42EF
:102AD00012D0C278120283789B189BB2C01884422D
:102AE00009D90378012B0ED94378022B0DD14379F4
:102AF000AB42EED100E0002070BD0020FCE70020DA
:102B0000FAE70020F8E70020F6E70020F4E7C046E7
:102B1000312A0000F8B50D001700884212D20024B7
:102B20000A4E03222900B04700280ED00378012B5B
:102B30000AD9A74209D00134E4B2C0188542F0D8BE
:102B4000002002E0002000E00020F8BD312A000053
:102B500010B506484030064B9847064B9847064844
:102B6000064B9847064B984710BDC04630030020DF
:102B700059290000DD22000008000020D1290000B2
:102B8000092A000010B5014B984710BD512B0000D9
:102B900070B500260C4D0D4C641BA410A64209D143
:102BA000002600F08FF80A4D0A4C641BA410A642C0
:102BB00005D170BDB300EB5898470136EEE7B3007E
:102BC000EB5898470136F2E7D02C0000D02C0000DB
:102BD000D02C0000D42C0000002310B59A4200D164
:102BE00010BDCC5CC4540133F8E703008218934253
:102BF00000D1704719700133F9E700002E2E2F68BD
:102C0000616C2F7372632F68616C5F75736172748E
:102C10005F73796E632E63002E2E2F68616C2F75A3
:102C200074696C732F7372632F7574696C735F6C46
:102C30006973742E630000002E2E2F68706C2F7342
:102C40006572636F6D2F68706C5F736572636F6D13
:102C50002E63000000200000AC02002000000000F5
:102C6000400000006C020020000000004000000056
:102C70002C0200200000000040000000F0280000AE
:102C8000D8250000F02800000A260000F0280000E7
:102C90002E250000F0280000F0280000F028000099
:102CA00042250000F02800003E2600002E2E2F7541
:102CB00073622F6465766963652F75736264632E32
:102CC00063000000F8B5C046F8BC08BC9E467047DB
:102CD000DD000000F8B5C046F8BC08BC9E46704751
:042CE000B50000003B
:102CE40000000000452000001000002065000020C6
:102CF4001201000202000040EB0304240001000062
:102D040000010902430002010080320904000001AD
:102D1400020200000524000110052401010004241E
:102D2400020205240600010705820340000A090483
:102D34000100020A00000007050102400000070527
:082D44008102400000000000C4
:00000001FF
